:020000040800F2
:1000000000020020F10400088D04000849040008E3
:100010009D040008AD040008BD04000800000000B5
:100020000000000000000000000000000D040008B7
:10003000CD04000800000000F1030008DD04000802
:100040008901000889010008890100088901000868
:100050008901000889010008691100086911000878
:100060006911000869110008691100088901000878
:100070008901000889010008890100088901000838
:100080008901000889010008890100088901000828
:100090008901000889010008890100086911000828
:1000A0008901000889010008890100088901000808
:1000B000011300088901000889010008890100086E
:1000C00089010008890100088901000889010008E8
:1000D0008901000889010008CD0E0008D30E000830
:1000E00069110008890100088901000889010008D8
:1000F00089010008890100088901000889010008B8
:100100008901000889010008071300088901000817
:100110008901000889010008890100088901000897
:100120008901000889010008890100088901000887
:100130008901000889010008890100088901000877
:100140008901000889010008890100088901000867
:100150008901000889010008890100088901000857
:100160008901000889010008890100088901000847
:1001700089010008890100088901000800000000C9
:10018000000000008901000800F0A8B900F0E8BAFA
:100190007047000070B50C46064600F045F9094B63
:1001A000094A1D682919914202D8084A914204D28D
:1001B0000C2333604FF0FF3500E0196000F03CF98C
:1001C000284670BD0002002000000220740B0020B1
:1001D0001946104600F0D0BA1946104600F0D4BABD
:1001E000132303604FF0FF307047132303604FF079
:1001F000FF307047132303604FF0FF307047022930
:100200004FF0000303608CBF002001207047000006
:10021000114B70B500241C60104B114D18682E68EE
:1002200000F09CF80F4B53F820301B68A3F1080234
:1002300096420FD026B13179092904BF0A213171C4
:10024000092103F8041C33F9021C074B2A601980AA
:10025000012070BD204670BD8C020020600300208C
:10026000940200209C02002090020020082930B552
:10027000037919D9082B32D842791A4B53F82250F6
:1002800000F108042DB12D68856053F822502C60D0
:1002900000E0846043F82240134C4279012303FAC2
:1002A00002F22368134319E0082B18D945790D4B46
:1002B00053F825203AB11468A2420BBF00222468EB
:1002C00043F825201460427953F822303BB9064C9C
:1002D000012303FA02F2236823EA02032360017177
:1002E00030BD00BF9C0200206003002008B50A4B0F
:1002F0001B681A79082A02D95B7983420AD900F06F
:100300009EF818B1054B01221A6008BDBDE80840EF
:1003100000F066B808BD00BF940200208C020020E7
:1003200008B500F081F8094B094A1B88094D1BB23A
:10033000002442F82340084A286813682146013BFC
:100340001360FFF793FF2C6000F046F89002002046
:10035000DC02002094020020980200200023C20743
:1003600002D440080133FAE718467047134423F0DB
:10037000030310B54FF077321C1F43F8042C6207BB
:1003800042BF4FF0883243F8082CA3F108044FF025
:10039000807304E909000F4B44F80C3C002344F837
:1003A000103C032344F8143C2246022344F8183C32
:1003B000012344F81C3C42F8201D0B2342F8043D65
:1003C000013B032BFAD120466FF0020340F8443D75
:1003D00010BD00BF2103000800F02AF801DFFEE78E
:1003E000024A536843F080535360704700ED00E0C9
:1003F000EFF3098020E9F00F40F804ED02490968A5
:10040000086000F003F8000094020020FFF700FFEE
:1004100004480068016801C9B1E8F00F81F3098858
:100420000047000094020020EFF3108072B670477E
:1004300062B6EFF31080704780F310887047EFF3D7
:100440000580C0B2704700000D490E4A0E4B684649
:10045000904203D8984201D9002102E009468D4616
:10046000012104207246024202D1EFF3088001E02C
:10047000EFF309802DE9F00F6B4600F06FF800BF35
:1004800000020020000002206005002008B502499B
:10049000042000F06DFA00BFD82F000808B502490B
:1004A000062000F065FA00BFE42F000808B50249F5
:1004B000072000F05DFA00BFF72F000808B50249D9
:1004C000082000F055FA00BF0930000808B50249BD
:1004D000092000F04DFA00BF1D30000808B50249A0
:1004E0000A2000F045FA00BF2F300008704770471F
:1004F00008B5FFF7FBFF6A46114B1249934202D23F
:1005000043F8041BFAE7104A104B11498B4204D2FE
:1005100052F8040F43F8040BF8E70E4B0E4A002183
:10052000934202D243F8041BFAE7FFF7E0FF00F022
:10053000FFF901F053F9BDE8084000F04BBA00BFE5
:1005400000000020FEE7FEE708350008000200205A
:100550008C0200208C020020740B00202DE9F04F4B
:100560009A46494B8FB093469A6B03925A6B04920A
:100570009F6ADA6A05921A6BDB6B0793434B06920C
:100580001A68434B9A420446884602D0414801F01B
:100590003BFAB8F1000F05D03F48002501F034FACE
:1005A0002E4626E094E80E00E068D4F81C900890EF
:1005B0002069099060690A9019F4007F3748A6699C
:1005C0000D930CBF04F1200504F124050C920B914E
:1005D00001F01AFA089B00930BA90EC9304801F0EC
:1005E00089F9CDF8009033460A9A09992D4801F00F
:1005F00081F92D4801F008FA39462C4801F07AF9C2
:1006000005992B4801F076F906992A4801F072F90C
:100610000799294801F06EF93A0403D50399274850
:1006200001F068F93B0603D50499254801F062F909
:10063000244801F0E9F95946234801F05BF9B8F183
:10064000000F1BD1214801F0DFF93146204801F0AD
:1006500051F969461F4BC91A03D549421E4801F09A
:1006600049F920468268C36801698C4641698E4613
:10067000AD46514691E8F00F4168006801BE174948
:10068000052000F075F900BF00ED00E0000000203B
:10069000FEE7FEE73D3000085330000882300008D6
:1006A0009D300008DA3000081831000821310008B8
:1006B0003131000841310008513100086131000832
:1006C0007131000881310008863100089831000836
:1006D000C931000858010020F13100081E3200081D
:1006E00010B568B1012815D1174A136823F0030328
:1006F0001360136843F4007343F0010313601BE0BD
:10070000114B1A6842F00E021A605A6842F4807265
:100710005A6011E00D4A136923F0040313610024A9
:10072000FFF782FEBFF34F8F30BFFFF785FE54B156
:10073000BDE8104000F06EBA044A136943F00403A8
:1007400013610124ECE710BD0070004000ED00E0F3
:1007500008B5FFF769FE0020BDE80840FFF7C0BFFD
:10076000034B044A4FF4E131002000F025BB00BFE9
:10077000040200208F0B00080A460146014800F0E1
:1007800011BA00BF0402002010B50A460C4601460B
:10079000002000F077FB204610BD002000F05ABD7D
:1007A000034B1968024611B9084600F033BD704783
:1007B000A8030020F0B51F4E1F4D33681F4C0133B6
:1007C00033601F4B00201A6818602B68226019469E
:1007D0000746B64641B1DEF800C08E68664503D8CC
:1007E0000F4601200968F5E700B1296007B9F0BD9F
:1007F00000213960E2B133B151685868814294BF39
:100800001146194600E01146084612681B680AB9ED
:1008100003600BE00BB9026008E055685E68B54202
:1008200094BF15461D4605602846EEE72160F0BDE1
:100830002360F0BDAC030020B4030020B00300200F
:10084000A40300202DE9F0412E4F2F4C01233B60E3
:1008500023683BB9FFF7AEFFFFF79FFF0130FBD0E6
:10086000002502E0FFF799FF05464FF000082368D6
:1008700023B9FFF792FF854214D91AE05E68FFF7AB
:100880008CFF854208D923685E68FFF786FFA8427F
:100890002CD3B042F7D329E08642F4D9361A132E6E
:1008A000E7D8F0E7236843B9FFF777FF85420646AC
:1008B0000BD9FFF77FFF0025D9E75E68FFF76DFFD3
:1008C000063E14308642D2D309E010F1140F04D34F
:1008D000FFF763FF8642FBD9EBE74FF0FF360023BB
:1008E0003B603046BDE8F041FFF75ABF23681A6805
:1008F0002260C3F80480C3F80880DA68186990475A
:10090000B5E700BFA8030020B003002008B500230E
:100910001846054A054900F0AFFC4FF0FF30BDE82E
:100920000840FFF73DBF00BF4508000840420F00E8
:1009300008B50121094800F01FFB0121084800F01B
:100940001BFB0121074800F017FB0121064800F0BE
:1009500013FBBDE8084000F011B900BF0D0C0240C8
:100960000C0C02400E0C02400F0C024070470000BD
:1009700008B50C4B1A680C4672B9012203281A609C
:1009800003D17146084800F0B5FF2146074800F042
:10099000B1FF074800F0AEFFFFF746FDFFF7E6FFA7
:1009A000FFF7D6FEB80300204332000847320008A4
:1009B0006332000808B500F051FD034800F09AFFCB
:1009C00000F0F2FC002008BD7132000808B500F00C
:1009D00003F9FCE71FB5FFF727FD0E4B0E481B6818
:1009E000029300240D4B00930F220C234FF48071CF
:1009F000019400F04DF80A4B0A481B6802930A4B19
:100A0000009307220C234FF4C061019400F040F8DA
:100A1000FFF7E2FC18020020BC030020CD0900080B
:100A20001C020020BC040020B509000808B5FFF72F
:100A3000FBFC094B1B681A79082A07D95A79074B1E
:100A400053F8221011B1096843F82210FFF7F4FCA3
:100A5000BDE80840FFF7C4BC940200209C020020BF
:100A600038B50B79082B03D908490320FFF780FF1D
:100A70004C7901F1080203682BB113F8035CAC4216
:100A800001D31846F7E78B60026038BD31320008A9
:100A90000F2A2DE9F74F05468B4691469A462AD8EC
:100AA00010F003031BBFC3F10403ED180B46CB1A70
:100AB000303B23F003031AF0080F05EB030405D0C5
:100AC0002A46A24203D212600432FAE72D60019353
:100AD000FFF7AAFC2749019B8046012251F82270AA
:100AE00016B25FB10132212AF8D14046FFF7A4FCCB
:100AF0006FF08A003BE06FF0150038E01D490C985C
:100B000041F822402A46E6800D99FFF72FFC0E9B04
:100B1000194AA3624FF0FF33E36113682060013389
:100B20001AF0010F6562C4F82CB084F805902771A3
:100B3000A760E76027616761A7612762136004D03F
:100B400001212046FFF792FB0DE00A212046FFF726
:100B50008DFB1AF0040F06D14046FFF76DFC4846A6
:100B6000FFF7C4FB02E04046FFF766FC304603B0E7
:100B7000BDE8F08FDC0200209802002008B500F0EC
:100B800009FE00F047F8BDE8084000F01CB838B591
:100B90000446043000F0CFFB0546204600F090FCF0
:100BA000284638BDF8B504460E461746051D3A4698
:100BB0003146284600F0AAFB20B90121204600F06A
:100BC0004FFCF4E7F8BD08B5002000F0A9F90120BA
:100BD000BDE8084000F0A4B9F8B50D4B1E68C6F397
:100BE00007221D4622B9F4B2003418BF012400E0E8
:100BF0000224FFF719FC2B689E42074602D12046CB
:100C0000FFF76EFD3846BDE8F840FFF715BC00BFA2
:100C10002002002038B5FFF707FC1B4C0023E360DF
:100C2000054600F037F84FF41443A360A268164B52
:100C300012F00C0FFAD1154A40F2057111608122B1
:100C40001A601A6842F480321A601A6812F4003F7F
:100C50000D4AFAD00E4B5360136843F08073136053
:100C60001168094B8901FBD59A6842F002029A602B
:100C70009A6802F00C02082AFAD100F017F8284608
:100C8000BDE83840FFF7D8BB00380240003C0240C6
:100C9000042A4007044B1A6842F001021A601A68DD
:100CA0009207FCD5704700BF00380240044B9A6899
:100CB00012F00C0F1EBF1A6822F001021A60704772
:100CC00000380240034B044A00280CBF1046184667
:100CD000704700BF00BD010580DE800204281CD8DB
:100CE000DFE800F003080D1217000D4B1A6C1143DA
:100CF000196412E00A4A536C194351640DE0084A22
:100D0000136B1943116308E0054A536B1943516390
:100D100003E0034A936B19439163BFF34F8F70470E
:100D200000380240042821D8DFE800F003090F153D
:100D30001B000F4A136C23EA0101116470470C4A2F
:100D4000536C23EA010151647047094A136B23EA8B
:100D5000010111637047064A536B23EA0101516395
:100D60007047034A936B23EA01019163704700BF08
:100D70000038024038B514230C4A4343D458256840
:100D8000AA0608D50A4B616803EBC002C9B253F842
:100D90003030506898472B0748BF6368054B1B6885
:100DA0001BB1BDE83840FFF741BE38BDCC3200086A
:100DB000BC0A00208C02002001282DE9F047804663
:100DC0000D46174603D92B490320FFF7D1FDDFF865
:100DD000B090294A142404FB009442F83070E6686D
:100DE00002EBC00201215360304600F0C5F83046E6
:100DF00000F098F93046617C00F05AF94E464FB148
:100E0000D4F808900021484600F0B6F8217C484606
:100E100000F04EF9142303FB08F806EB080999F8D3
:100E200012A0D9F804105046FFF758FF56F80840B2
:100E30000023E360504623616361FFF743FFB0FB8B
:100E4000F5F080B2A06077B199F8133001215AB261
:100E500003F01F0301FA03F35209084941F8223055
:100E600042F22C0301E042F20803E3600020BDE8F7
:100E7000F08700BF31320008BC0A002000E100E02A
:100E8000CC320008012838B505D80E4C14230A448A
:100E900003FB004309E00C490320FFF769FD2568C7
:100EA0002D06FCD511F8015B65608A4201D01C68F3
:100EB000F5E714235843034B1A5813685B06FCD517
:100EC00038BD00BFCC320008313200080020FFF7E7
:100ED00051BF0120FFF74EBFF8B5104C04EB401492
:100EE00001216768384600F047F8A66800213046BF
:100EF00000F042F8E5680121284600F03DF8247D25
:100F00003846214600F0D4F82146304600F0D0F8AB
:100F100021462846BDE8F84000F0CAB8F43200087F
:100F200001282DE9F041044603D910490320FFF7B9
:100F30001FFD0F4BDFF83C80002543F82050640173
:100F4000FFF7CAFF08EB04031E7F9F69304639464E
:100F5000FFF7C4FE58F8043039461D603046DD61A5
:100F60005D60BDE8F041FFF7DDBE00BF3132000833
:100F7000CC0A0020F4320008F8B50D460126C0F373
:100F8000832120F00F0400F00F0706FA01F1022080
:100F9000FFF7A4FE07FA06F00323216883406FEAF7
:100FA000030C01EA0C012160216805F0030E0EFA22
:100FB00000FE4EEA01012160E2680CEA0202E260F2
:100FC000E168C5F3810282400A43E2606268BE4084
:100FD00022EA060666606268C5F30015BD40154347
:100FE0006560A2681343A3600020F8BD2DE9F041BD
:100FF00000F00F0415462B4A42F8343002EBC402CD
:10100000069B536006468846C0F383274FF4804111
:101010000120FFF763FE41463046FFF7ADFF042C89
:10102000214B03DCA11D01228A4003E0092C03DCD3
:101030004FF400021A6002E04FF480725A601B4BBA
:101040000120996800FA04F2D2431140996099682E
:1010500005EA000E0EFA04FE4EEA01019960D96815
:101060000A40DA60C540DA68A54004F00C0404F1D7
:10107000804404F59C341543DD6006F00302A56846
:1010800092000F21914025EA0101A160A1689740DB
:10109000B0400F43A76058611A68104318600020E1
:1010A000BDE8F081D40A002000E100E0003C0140EE
:1010B00020F00F0300F00F02F0B51E685700032563
:1010C000BD4026EA05051D601D680224072A04FAB2
:1010D00007F444EA050494BF002201221C6003EBDC
:1010E000820300F007001C6A80000F22824024EA7D
:1010F00002021A621A6A814041EA02001862F0BDD7
:1011000020F00F0300F00F00196810B5032244000F
:10111000A2400A4214BF5B691B69012202FA00F077
:10112000184010BD20F00F02012300F00F0003FA59
:1011300000F09061704720F00F0200F00F001030B7
:10114000012303FA00F09061704710B50446FFF7E1
:10115000D7FF20B12046BDE81040FFF7ECBF204686
:10116000BDE81040FFF7DEBF104B2DE9F0415E698E
:101170001A680F4F164000244FF001081D4608FA68
:1011800004F31E4206D06B6107EBC40357F834200A
:10119000586890470134102CF1D1064B1B681BB1E5
:1011A000BDE8F041FFF742BCBDE8F081003C0140E2
:1011B000D40A00208C0200202DE9F843124ADFF8FF
:1011C000508003010746D5582E69EB6800241E4065
:1011D00008EBC0090223A3401E4209D0EA68D9F8EF
:1011E000040022EA0303EB60214658F837309847A1
:1011F0000134042CEED1054B1B681BB1BDE8F8434C
:10120000FFF714BCBDE8F883343300088C020020DB
:10121000540B0020032910B516D80D4B00011C18E3
:101220001B586068024001F10C0003EB8000426033
:101230001869022202FA01F120EA01021A61DA6851
:101240001143D960002010BD4FF0FF3010BD00BF2A
:10125000343300080001024B1B58586A704700BF26
:1012600034330008034B00011A58136843F001039C
:10127000136070473433000801282DE9F843054610
:10128000884630D81A4E1B490401371941F83020DE
:1012900097F80C9001EBC00148464B60B968FFF726
:1012A0001DFD36597B680024346048467460F36243
:1012B000FFF708FD104B7A7B13F809305843B0FB59
:1012C000F8F3013BB36251B2012302F01F027361D4
:1012D00049099340094A284642F82130FFF7C2FFE6
:1012E0002046BDE8F8834FF0FF30BDE8F88300BF2B
:1012F00034330008540B00205433000800E100E0B0
:101300000020FFF759BF0120FFF756BF70B5134605
:101310007BB18568C468A5420BD084680668651CEB
:1013200085604568013D2C40013B345D01F8014B6F
:10133000EEE7D01A70BDC368426830B584681B1BE5
:10134000934208D0C3680468013A5D1C1340C5602D
:10135000E154002030BD4FF0FF3030BD37B50E4DA9
:101360002B68002003F16404FFF774FF844211D25C
:101370000A4800F0BFFA0A48FFF7E7FE094B0024CD
:10138000B3F900100194684600F0DEF92046FFF73B
:1013900061FF286003B030BD680B002056330008A1
:1013A0000C0C0240640B002030B51E4885B000F0E4
:1013B000A1FA01211C48FFF7DFFD002801DA1B48D4
:1013C0000FE01B4800F096FA1748FFF7B4FE1948E3
:1013D0000090194B01220821FFF708FE002805DACA
:1013E000164800F011FB012005B030BD1448154D22
:1013F000154C00F07FFA0020FFF72CFF134B18600C
:10140000134B1A88134B1A8002A800F0BFF9064844
:10141000FFF776FE002814BF294621460E4800F04B
:1014200069FAF1E76C3300080C0C02408E330008B7
:10143000BB330008000002405D130008E8330008D9
:10144000243400086533000868330008680B002066
:1014500090020020640B002049340008FFF756BAC0
:1014600070B505460C46FEF7DFFF2B6806462BB924
:101470004FF0FF332B60FEF7DFFF18E0CCB10F4BCE
:101480001C6802212046FEF7F1FE2B68013305D1CE
:1014900004F108032B600023A36003E021462846E3
:1014A000FFF7DEFA3046FEF7C7FFFEF799FF01208F
:1014B00070BDFEF7C1FF204670BD00BF9402002042
:1014C00070B50446FEF7B0FF256806461DB16B1CDB
:1014D00005D100232360BDE87040FEF7ADBF28466C
:1014E0000A2150F808392360FEF7C0FE236813B9BB
:1014F0004FF0FF33236015F8034C3046FEF79CFF96
:101500002046BDE87040FEF7F1BE0000F8B5054684
:101510000E46FEF789FF364B364A1B881BB207463C
:1015200052F82320D2F820E0BEF1000F1AD05469FF
:101530009369A34216D9631C5361D3691C4046B911
:10154000136933B9631C04D13846FEF775FF204692
:10155000F8BD002C0ADB0EEBC40393E8030085E81A
:10156000030004E04FF0FF34002EE9D0D560166987
:1015700076B333681361002C0CDB95695169D3692C
:10158000691A8B42A9BF691C4FF0FF351D4091615C
:101590000EEBC505736893E8030085E8030016F8B1
:1015A000043C052B09D0002373600A21A6F1080032
:1015B000FEF75CFE16F8034C00E00F243846FEF7F9
:1015C0003BFF0E2C02D82046FEF790FE0120F8BD0E
:1015D000002C09DA10460321FEF748FE3846FEF7D4
:1015E0002BFFFEF7FDFEF1E73846FEF725FFEDE79E
:1015F00090020020DC02002010B583694469C269B2
:101600001C1BA24201DA002010BD5C1C1340846147
:10161000F9D4026A03C902EBC30383E80300012083
:1016200010BD00002DE9F8431E46264B53F821500B
:10163000254B1B880380074691462DB93046FEF79F
:10164000FBFE4FF0FF3439E02B79032B28D01F4BE2
:1016500001462846D3F80080FFF7CEFF044638B194
:101660003046FEF7E9FE98F80430052B25D122E03C
:10167000B9F1000F03D13046FEF7DEFE1EE098F808
:101680000430C8F80C70052B0CBF0521042140461E
:10169000FEF7ECFD414605F11000FFF7E1F907E028
:1016A00003C8EB6883E803000A212846FEF7DEFD45
:1016B0003046FEF7C1FEFEF793FE01242046BDE84A
:1016C000F88300BFDC02002090020020940200207A
:1016D00038B50446FEF7A8FE074B1B882380074B4E
:1016E000214605461868FFF787FF04462846FEF79F
:1016F000A3FE204638BD00BF9002002094020020C7
:1017000008B50F4B53F82130B3B1212202801A796A
:10171000032A0BD103C8DA6882E8030018460A21BD
:10172000FEF7A4FD074B0120186008BD01461846CE
:10173000BDE80840FFF760BF4FF0FF3008BD00BFB5
:10174000DC0200208C02002070B504460D46FEF736
:1017500076FE28B129462046BDE87040FFF7D0BF8D
:10176000094B1B881BB29D4204D12046BDE8704046
:10177000FFF7AEBFFEF758FE29460346012220467A
:10178000BDE87040FFF74EBF900200200121FFF737
:10179000BDBE00000F4BD3F8882042F47002C3F89E
:1017A00088200D4A9A60102283F822200021DA77DF
:1017B00001F1604000F561400131522980F80023B9
:1017C000F6D11A6942F010021A615A6942F40072A5
:1017D0005A61704700ED00E00000000870B50F4E40
:1017E0000F4D761BB61018BF002405D0013455F8F4
:1017F000043B9847A642F9D10A4E0B4D761BFEF7E3
:10180000C5FCB61018BF002406D0013455F8043BBF
:101810009847A642F9D170BD70BD00BF0C350008D5
:101820000C3500080C3500080C35000870B484072E
:1018300046D0541E002A41D0CDB2034602E0621EBB
:10184000E4B3144603F8015B9A07F8D1032C2ED9B0
:10185000CDB245EA05250F2C45EA054519D903F116
:1018600010022646103E0F2E42F8105C42F80C5C27
:1018700042F8085C42F8045C02F11002F2D8A4F1CC
:10188000100222F00F0204F00F041032032C134454
:101890000DD91E462246043A032A46F8045BFAD8BC
:1018A000221F22F003020432134404F003042CB17B
:1018B000C9B21C4403F8011BA342FBD170BC7047A2
:1018C00014460346C2E700BF0EB410B5044683B009
:1018D00018B183690BB900F04DFB06A803460190CF
:1018E000059AA168204600F007FD03B0BDE810404E
:1018F00003B070470FB410B50A4B1C6882B024B116
:10190000A36913B9204600F035FB05A803460190F2
:10191000049AA168204600F0EFFC02B0BDE8104038
:1019200004B07047240200202DE9F0410E468046A5
:1019300000283ED08369002B39D084682F4B9C420D
:1019400043D02F4B9C4256D02E4B9C4208BFD8F818
:101950000C40A3891B073DD52369002B3AD0013EDB
:10196000A36816F8015F013BA360B5B1002B04DB4F
:1019700023685A1C22601D70F2E7A769BB42224609
:101980002946404601DB0A2DF2D100F045F801302E
:10199000E6D14FF0FF30BDE8F081002B21DB23685A
:1019A0000A22591C21601A701046BDE8F08100F02F
:1019B000E1FAD8F81830D8F80840002BBED14046DC
:1019C00000F0D8FA0D4B9C42BBD1D8F80440A38953
:1019D0001B07C1D42146404600F080F80028BED045
:1019E000D7E7224640460A2100F016F80130D0D051
:1019F0000A20BDE8F081D8F80840AAE7B034000812
:101A00009034000870340008024B01461868FFF754
:101A10008BBF00BF24020020F8B50E4614460546D1
:101A200010B18369002B41D0254B9C4243D0254BFC
:101A30009C4242D0244B9C4208BFEC68A389A26917
:101A4000A2601A0721D52369FBB122686169D31A04
:101A50008B42F7B221DA0133A168501C0139A16031
:101A60002060167062699A4206D0A389DB0701D50F
:101A70000A2F01D03846F8BD2146284600F040F92B
:101A80000028F7D04FF0FF37F4E72146284600F052
:101A900025F80028F6D12369D7E72146284600F02B
:101AA0002FF90028EED122680123D5E700F062FA71
:101AB000034B9C42BBD16C68C0E7AC68BEE700BF7B
:101AC000B03400089034000870340008024B0A4615
:101AD00001461868FFF7A0BF24020020384B70B5FC
:101AE0001D6806460C4615B1AB69002B42D0354B3C
:101AF0009C4245D0344B9C4258D0344B9C4208BF4A
:101B0000EC68B4F90C2093B219070CD52069A8B180
:101B100013F001021ED0636900225B42A361A26040
:101B2000F0B1002070BDDD0642D558072AD42069E7
:101B300042F00803A3819BB20028E9D103F420728C
:101B4000B2F5007FE4D03046214600F0B1FAA38917
:101B50002069DDE7990758BF6269A2600028E0D1DB
:101B6000B4F90C301A06DDD543F04003A3814FF0E1
:101B7000FF3070BD284600F0FDF9124B9C42B9D1F0
:101B80006C68BEE7616B51B104F14403994204D023
:101B9000304600F0D1FAB4F90C200023636300232F
:101BA0002069636022F024022060C1E7AC68A8E7E6
:101BB00042F04002092333604FF0FF30A28170BD34
:101BC00024020020B034000890340008703400086B
:101BD0008B891A072DE9F0410D46804635D44A68B5
:101BE000002A6BDDEC6A002C47D003F48052002100
:101BF00092B2D8F80060C8F80010002A62D06A6D6E
:101C00005F0705D569686B6B521A0BB12B6CD21A42
:101C10000023296A4046A047441C39D0AB892A6971
:101C20002A60DB044FF000026A6045D4696BC8F893
:101C3000006011B305F14403994202D0404600F020
:101C40007BFA00206863BDE8F0810E69AEB10C68D4
:101C50000E6098070CBF4B690023A41B8B600AE041
:101C600023463246AF6A296A4046B8470028A4EBAB
:101C70000004064404DD002CF2DC0020BDE8F08105
:101C8000AB8943F04003AB814FF0FF30BDE8F081FA
:101C9000D8F800201D2AF3D8184BD34003F00103D5
:101CA00083F00101002BEBD0AB892C696960D9046A
:101CB0002C60BBD5002AB9D16865B7E70A6C002A49
:101CC00090DCDAE70123296A4046A047431C02461C
:101CD00002D0AB89EC6A93E7D8F80030002BF8D03B
:101CE0001D2B01D0162B02D1C8F80060C5E7AB89C7
:101CF00043F04003AB81BDE8F08100BF010040200C
:101D00000B6933B310B5044682B008B18369ABB137
:101D1000114B994219D0114B994218D0104B99424E
:101D200008BFE168B1F90C3013B9002002B010BD52
:101D3000204602B0BDE81040FFF74ABF019100F015
:101D400019F90199044B9942E5D16168EAE7A16864
:101D5000E8E70020704700BFB03400089034000866
:101D60007034000820B1054B01461868FFF7C8BF62
:101D7000034B0449186800F043B900BF2402002057
:101D800068340008011D000800207047014900F078
:101D900037B900BF011D00080020704770B56823E7
:101DA0004D1E03FB05F50E4605F1740100F00AFA1D
:101DB000044640B100210C30666005F168022160E4
:101DC000A060FFF733FD204670BD00BF1F4B70B50C
:101DD0001D68AB69064613B9284600F039F8483546
:101DE0006B68AC68013B05D521E0013B5A1C04F14E
:101DF00068041CD0B4F90C20002AF6D10025012378
:101E00004FF6FF72E281A38165662560A56065607B
:101E100025616561A5612946082204F15C00FFF790
:101E200005FD6563A563A564E564204670BD2B6868
:101E30000BB11D46D4E704213046FFF7AFFF286001
:101E400008B10546CCE70C23336070BD6834000848
:101E50003D4B3E491A682DE9F04F90424FF0000388
:101E60008364C364036508BF012383B008BF836133
:101E700081620746FFF7AAFF78603846FFF7A6FFA2
:101E8000B8603846FFF7A2FF7D68F860002404239D
:101E9000AB812C606C60AC606C66EC812C616C6119
:101EA000AC61214605F15C000822FFF7BFFCBE686B
:101EB000DFF89CB0DFF89CA0DFF89C90DFF89C80F6
:101EC000C5F824B001230922C5F828A0C5F82C9034
:101ED000C5F830802D622146F381B2813460746090
:101EE000B460746634617461B46106F15C00082208
:101EF0000193FFF79BFCFD68366212200222C6F8B0
:101F000024B0C6F828A0C6F82C90C6F83080214628
:101F1000A881EA812C606C60AC606C662C616C619D
:101F2000AC6105F15C000822FFF780FC019B2D628B
:101F3000C5F824B0C5F828A0C5F82C90C5F83080A5
:101F4000BB6103B0BDE8F08F683400088D1D000848
:101F50005129000879290008B5290008D529000869
:101F6000024B0349186800F04BB800BF6834000802
:101F7000011D0008836903B96AE77047704700BF15
:101F8000704700BF704700BF704700BF024B034956
:101F9000186800F00FB800BF24020020991D000847
:101FA000024B0349186800F005B800BF2402002066
:101FB000891D00082DE9F04110F148071BD0884623
:101FC00000267D68BC68013D0FD4A389012B05F173
:101FD000FF3506D9B4F90E300133204601D0C04791
:101FE00006436B1C04F16804EFD13F68002FE8D171
:101FF0003046BDE8F0813E463046BDE8F08100BF86
:102000002DE9F84310F148071FD0884606464FF0E7
:1020100000097D68BC68013D11D4A389012B05F13D
:10202000FF3508D9B4F90E3001332146304602D0CD
:10203000C04749EA00096B1C04F16804EDD13F6810
:10204000002FE6D14846BDE8F883B9464846BDE8CA
:10205000F88300BF70B50C46B1F90E10002990B09E
:1020600015461E4613DB01AAFEF7C4F800280EDB56
:10207000029A02F47042A2F50052B2FA82F25209B8
:102080004FF48063002032602B6010B070BDA389D4
:1020900000221B06326004D5402300202B6010B0C4
:1020A00070BD4FF4806300202B6010B070BD00BF86
:1020B0008A8992070B4606D501F1470201211A6071
:1020C0001A6159617047F0B583B001AB6A460C469E
:1020D0000546FFF7BFFF00990646284600F072F854
:1020E000B4F90C30D0B1019A124F0099AF6243F0AD
:1020F0008003A3812060206161611AB93343A38109
:1021000003B0F0BD2846B4F90E10FEF778F8B4F924
:102110000C300028F2D043F00103EFE79A05EFD42A
:1021200004F1470243F002030121A38122602261EE
:102130006161E5E78D1D000830B481B151F8043CC0
:102140000439002BB8BFC9181D4B1A682AB18A423E
:102150000AD908680C18A24225D04A60196030BC20
:1021600070478B4203D81A465368002BF9D1146884
:1021700015198D420CD007D808680C189C4218D04D
:102180004B6030BC516070470C23036030BC70471B
:1021900009680C44111999421460E0D10ACB0C442F
:1021A00053601460DBE7146852684A60204408609A
:1021B000D4E71C685B684B60204408605160CEE740
:1021C0006C0B002070B5CD1C25F0030508350C2DD7
:1021D00038BF0C25002D06463BDBA94239D82749DC
:1021E0000A6852B113685B1B04D436E023685B1B9A
:1021F0001AD522465468002CF8D149681F4C002992
:1022000036D029463046FDF7C5FF431C21D0C41CFB
:1022100024F00304A04205D0211A3046FDF7BAFF8E
:10222000013016D0256004E00B2B0DD923601C442F
:10223000256004F10B0020F00700231DC31A02D013
:102240005A42E25070BD70BD94420ED06368536034
:10225000EFE70C233360002070BD0B2B03D85368CD
:1022600014460B60E5E71446E0E713461446F8E72A
:102270003046FDF78FFF6060C3E700BF6C0B0020A6
:102280009368013B002B10B4936007DBCCB213685A
:10229000581C10601970204610BC70479469A34206
:1022A00002DBCCB20A2CF2D110BCFFF7B5BB00BFE9
:1022B00093B1F8B514460F460646D51801E0AC4276
:1022C00008D03A4614F8011B3046FFF7D9FF431CEB
:1022D000F5D1F8BD0020F8BD00207047936810B517
:1022E000144613B95360184610BD00F077FB002365
:1022F000A360636010BD00BF2DE9F04F9DB088461C
:1023000014460393814618B18369002B00F00B81BA
:102310008B4B984500F00D818A4B984500F00C815D
:10232000894B984508BFD9F80C80B8F80C301D07C8
:1023300040F1EF80D8F81030002B00F0EA80302315
:102340008DF82A302378814DDFF804A20021202265
:1023500009918DF82920002B00F08580252B264639
:1023600003D117E0252B00F0868016F8013F002BE3
:10237000F8D1B6EB040B76D022465B464146484680
:10238000FFF796FF01306ED0099B32785B440993CA
:10239000002A68D000234FF0FF31721C049307938A
:1023A00006938DF853301A930591012604E00499A1
:1023B00006FA03F30B43049314466448217805227C
:1023C00000F08EFC621C431B0028F0D1049BD80651
:1023D00044BF20228DF853201907217844BF2B22B7
:1023E0008DF853202A2968D0A1F13002092A0BD890
:1023F000079B14F8011F03EB830302EB4303A1F1D6
:102400003002092AF5D907932E293FD003225048DC
:1024100000F066FC48B10499CAEB0000402202FAC1
:1024200000F041EA000301340493217849488DF813
:1024300028100622013400F053FC00285FD0464BE0
:10244000EBB103AB00934246444B04A94846AFF3BB
:10245000008007467A1C06D0099B3B4409932378E9
:10246000002B7FF47BAFB8F80C305B0658D409988A
:102470001DB0BDE8F08FB6EB040B8BD07CE7039B5F
:10248000073323F0070308330393E5E761782A292C
:102490001DD0A1F130020023092A04F101040593A3
:1024A000B4D814F8011F03EB830302EB4303A1F13B
:1024B0003002092AF5D90593A8E7039A1168043276
:1024C0000029039215DB0791617801349CE7039B97
:1024D0001A680592002A03F104030393B8BF4FF072
:1024E000FF3204F10203AEBFA178A17805921C4629
:1024F0008CE7494243F0020307910493E4E703ABFE
:1025000000934246154B04A9484600F0CDF8074613
:10251000A0E741464846FFF7E1FA00283FF40FAF35
:102520004FF0FF30A4E7FFF725FD054B98457FF4FA
:10253000F3AED9F80480F8E6D9F80880F5E600BFD4
:10254000B03400089034000870340008D03400081B
:10255000D8340008DC34000800000000B122000874
:1025600010B4044C13460A460146206810BCFFF71D
:10257000C3BE00BF240200202DE9F0470C4691465F
:102580000969A268DDF820808A42B8BF0A46C9F806
:10259000002094F8431006461F4611B10132C9F8D5
:1025A0000020236899065DD5D9F800200232C9F8C9
:1025B0000020236813F0060F19461DD1E1688A1A1E
:1025C000002AD8BF194617DD04F1190A002505E0D5
:1025D000E368D9F800209B1AAB420CDD0123524678
:1025E00039463046C047013005F10105F0D14FF0C2
:1025F000FF30BDE8F087216894F84330003318BFFE
:1026000001238A060AD5E1185A1C302081F84300BC
:10261000224494F8451082F84310023304F1430237
:1026200039463046C0470130E1D0236803F0060345
:10263000042B29D0A36822699342C8BF4FF0000938
:102640002FDD9B1A99441A34002501E04D4528D00E
:102650000123224639463046C047013005F10105C5
:10266000F4D1C4E713F0060F08D1E168D9F80020CF
:102670008A1A002AD8BF1946A6DCBDE794F8433071
:10268000003318BF0123C9E7D9F80000E168A36847
:102690002269091A934221EAE179D2DCB9F1000FEB
:1026A000D1D10020BDE8F0872DE9F0430C46097E2A
:1026B00085B06E29064617460C98984604F1430CDF
:1026C0005AD01AD8632900F0128100F2D68000296E
:1026D0005CD0582940F0F58084F8451022680368E2
:1026E000DFF864E2150603F104011ED4550653BF5A
:1026F0001B6801601B88016019E0732900F0CF801E
:102700007ED86F2900F0E480702940F0DA802268DA
:1027100042F020022260782384F845300368DFF815
:102720002CE2150603F10401E0D51B680160D00717
:1027300044BF42F020022260002B40F090802268CB
:1027400022F0200222601021002284F843206068D9
:10275000A0600028C0F28880226822F00402226073
:10276000002B62D1002840F08180654608296AD09C
:10277000C5EB0C0323610CE023681A0640F1D580F9
:1027800003686269191D01601B681A6000236546B1
:102790002361CDF800803B4603AA21463046FFF76F
:1027A000EBFE013021D02A46236939463046C04726
:1027B00001301AD02368039813F0020FE36819D090
:1027C0001A1A002A16DD04F11909002504E0E3684D
:1027D00003981A1AAA420DDD01234A4639463046AB
:1027E000C047013005F10105F1D14FF0FF3005B0D0
:1027F000BDE8F0839842B8BF184605B0BDE8F08345
:10280000752965D078295CD1226884E76168A16068
:102810002D200029C3F1000384F8430021DB22F0BE
:102820000402DFF824E122600A216546B3FBF1F2DD
:1028300001FB123013461EF8002005F8012D002B75
:10284000F4D1082994D12368D90791D56268236906
:102850009A428DDC302305F8013C013D88E71021C8
:1028600072E7DFF8E4E00A21002BDED19EF80030A9
:1028700084F8423004F1420578E7642901D06929DF
:102880001FD122680368150603F104013AD51B68BD
:102890000160002BBADBDFF8B0E00A2157E70368DC
:1028A0006268191D01601D680021284600F018FAB1
:1028B000002846D0401B60602061002384F843302C
:1028C00067E7012384F84210236104F14205F4E72D
:1028D00023681A061ED503681A1D1B680260227E33
:1028E000DFF864E06F2A14BF0A2108212CE703688F
:1028F0001A68191D0123016004F1420584F8422081
:102900002361DAE7550653BF1B680160B3F9003055
:102910000160BEE713F0400F036803F1040215BF26
:1029200002601B681B880260D9E713F0400F036840
:10293000626903F1040101601B6814BF1A801A6008
:1029400024E76068B8E700BFE4340008F834000802
:1029500010B50C46B1F90E10FDF73AFC002803DB68
:10296000636D0344636510BDA38923F48053A38181
:1029700010BD00BF002070472DE9F0411646B1F9A7
:102980000C201F46D3050C46054607D5002202231E
:10299000B1F90E10FDF729FCB4F90C20B4F90E10B2
:1029A00022F48052A2813B4632462846BDE8F041DF
:1029B000FDF712BC10B50C46B1F90E10FDF715FC71
:1029C000A389421C0EBF23F4805343F480536065F7
:1029D000A38110BDB1F90E10FDF702BC9368002B66
:1029E00076D02DE9F04F8B8985B00C461907019000
:1029F000164629D522693AB303F002081FFA88F077
:102A0000356800282FD04FF00009B44FC846B246B1
:102A1000B84543464A4628BF3B460198B8F1000FE7
:102A200050D0216AA66AB047002871DDDAF8083074
:102A30001B1A8144C0EB0808CAF80830002BE7D104
:102A4000002005B0BDE8F08F21460198FFF746F859
:102A5000002840F03A81A389356803F002081FFA84
:102A600088F00028CFD113F001095BD14F460296C0
:102A70001FB39A05D4F808802CD54745C246C0F04C
:102A8000A48013F4906F40F0B1802068524649460C
:102A900000F010FAA0682368C8EB00005344A0605F
:102AA00023603846029A93681B1A81443F1A936048
:102AB000002BC5D0A389002FDBD1D5F800906F681B
:102AC0000835D5E7D5F80090D5F8048008359FE79C
:102AD0000020704720682369984203D861698F42BB
:102AE00080F0B780B84528BFB8464246494600F056
:102AF000E1F9A3682268C8EB03034244A3602260A3
:102B0000002B49D121460198FFF7FAF8002843D05D
:102B1000B4F90C3043F040034FF0FF30A38105B00F
:102B2000BDE8F08F8046029082468146B9F1000FE1
:102B30002AD0029B002B4CD0206823696269C845CB
:102B4000C34628BFCB4698425F4604D9A3681344C6
:102B50009B4500F39080934520DB1346A76A216ACA
:102B600001985246B847071ED2DDB8EB070823D0BC
:102B7000B368DB1BBA44C7EB0909B360002B3FF411
:102B80005FAFB9F1000FD4D10023D5F800A0D5F87C
:102B9000049002930835C9E7404683E75A465146F8
:102BA00000F088F9A2682368CBEB02025B44B8EB23
:102BB0000708A2602360DBD121460198FFF7A0F847
:102BC0000028A5D1CDF80880D2E72068B846BA46DB
:102BD0005CE74A460A21504600F082F800286FD090
:102BE00001300123CAEB00080293A5E7626920685F
:102BF000216902EB4208C1EB000A08EBD8780AF120
:102C000001004FEA680838444045424684BF804688
:102C100042465B0542D511460198FFF7D3FA834639
:102C2000002855D05246216900F0AAF8A38923F460
:102C3000906343F08003A381CAEB08030BEB0A0007
:102C4000C4F81480C4F810B02060A360B846BA4637
:102C50001CE76FF00043BB4228BF3B464A4693FB4C
:102C6000F1F30198A66A01FB03F3216AB04700283B
:102C70003FF718AF4CE71A465146039300F01AF994
:102C80002268039B01981A4422602146FFF738F816
:102C9000039B00287FF43CAF1F4666E7019800F0D5
:102CA0006DF983460028C7D1019D21692846FFF7A9
:102CB00043FAB4F90C300C2223F080032A6029E790
:102CC000012309F10108029336E74FF0FF30B8E61F
:102CD000019A0C231360B4F90C301BE700FCFF7F52
:102CE00001F0FF01102A2BDB10F0070F08D010F8BD
:102CF000013B013A8B422DD010F0070F42B3F6D1C1
:102D0000F0B441EA012141EA014122F007047FF0D9
:102D100000070023F0E80256083C85EA010586EA30
:102D2000010685FA47F5A3FA87F586FA47F6A5FA6C
:102D300087F68EB9EED1F0BC01F0FF0102F0070278
:102D400032B110F8013B013A83EA010313B1F8D123
:102D50000020704701387047002D06BF3546033804
:102D6000073815F0010F07D1013015F4807F02BF3D
:102D7000013015F4C03F0130F0BC0138704700BF8E
:102D8000844641EA000313F003036DD1403A41D376
:102D900051F8043B40F8043B51F8043B40F8043B35
:102DA00051F8043B40F8043B51F8043B40F8043B25
:102DB00051F8043B40F8043B51F8043B40F8043B15
:102DC00051F8043B40F8043B51F8043B40F8043B05
:102DD00051F8043B40F8043B51F8043B40F8043BF5
:102DE00051F8043B40F8043B51F8043B40F8043BE5
:102DF00051F8043B40F8043B51F8043B40F8043BD5
:102E000051F8043B40F8043B51F8043B40F8043BC4
:102E1000403ABDD2303211D351F8043B40F8043B64
:102E200051F8043B40F8043B51F8043B40F8043BA4
:102E300051F8043B40F8043B103AEDD20C3205D374
:102E400051F8043B40F8043B043AF9D2043208D06C
:102E5000D2071CBF11F8013B00F8013B01D30B88DE
:102E600003806046704700BF082A13D38B078DD0BC
:102E700010F003038AD0C3F10403D21ADB071CBF8E
:102E800011F8013B00F8013B80D331F8023B20F8F8
:102E9000023B7BE7043AD9D3013A11F8013B00F831
:102EA000013BF9D20B7803704B7843708B788370B9
:102EB000604670478842F0B50DD98B1898420AD207
:102EC0008118002A51D09A1A13F8014D01F8014DCA
:102ED0009342F9D1F0BD0F2A48D941EA00039B077C
:102EE00046D100F1100401F11003154653F8106C9F
:102EF00044F8106C53F80C6C44F80C6C53F8086CE4
:102F000044F8086C103D53F8046C44F8046C0F2D21
:102F100003F1100304F11004E8D8A2F1100323F028
:102F20000F0302F00F0E1033BEF1030F19440344D8
:102F300021D91E1F0D467446043C55F8047B46F803
:102F4000047F032CF8D8AEF1040424F00304043405
:102F50002344214402F0030262B1013B0A4411F808
:102F6000014B03F8014F8A42F9D1F0BD0346F3E764
:102F70000346F2E7F0BD7246EEE700BFF9B1F8B5DF
:102F800006461546B2B10C4600F01CF8854201D841
:102F90002046F8BD29463046FFF714F9074668B1C8
:102FA0002A462146FFF7ECFE30462146FFF7C4F8DB
:102FB0003846F8BDFFF7C0F82846F8BDF8BD114601
:102FC000FFF700B951F8040C0028BEBF091851F8EA
:102FD000043CC018043870474E4D492048414E44C7
:102FE0004C4552004D454D204D414E4147452048EE
:102FF000414E444C455200425553204641554C5495
:103000002048414E444C45520055534147452046C7
:1030100041554C542048414E444C45520044454291
:103020005547204D4F4E2048414E444C4552004498
:10303000554D4D592048414E444C4552000A495384
:103040005220737461636B206F766572666C6F7764
:10305000656400537461636B20706F696E74657290
:1030600020636F727275707465642C20726573656D
:103070007420746F20746F70206F662073746163A6
:103080006B000A436F6E74657874206265666F72B8
:103090006520686172646661756C743A0020202056
:1030A00072303A2030782530386C780A202020722F
:1030B000313A2030782530386C780A20202072325E
:1030C0003A2030782530386C780A20202072333A44
:1030D0002030782530386C780A0020207231323A5E
:1030E0002030782530386C780A2020206C723A2005
:1030F00030782530386C780A20202070633A2030F0
:10310000782530386C780A20207073723A20307835
:103110002530386C780A0A004653522F4641523AFD
:103120000020434653523A2030782530386C780AD4
:103130000020484653523A2030782530386C780ABF
:103140000020444653523A2030782530386C780AB3
:103150000020414653523A2030782530386C780AA6
:103160000020424641523A2030782530386C780AA7
:10317000004D4D4641523A2030782530386C780A5F
:10318000004D697363004558435F5245543A2030FF
:10319000782530386C780A00417474656D707469F4
:1031A0006E6720746F207265636F6E7374727563DF
:1031B0007420737461746520666F72206465627533
:1031C0006767696E672E2E2E00496E204744423A8B
:1031D0000A2020736574202470633D3078256C7854
:1031E0000A20206672616D6520300A202062740A10
:1031F000000A49535220737461636B206F766572C5
:10320000666C6F776564206279206174206C6561FB
:1032100073742025642062797465732E0A00484116
:103220005244204641554C542048414E444C45524E
:10323000004641494C454420415353455254494F5F
:103240004E2E0025700A002A2A2A2052494F542067
:103250006B65726E656C2070616E69633A0A2573E6
:103260000A0A002A2A2A2068616C7465642E0A0AF8
:10327000006D61696E28293A20546869732069736A
:103280002052494F5421202856657273696F6E3A57
:1032900020554E4B4E4F574E20286275696C646422
:1032A00069723A202F686F6D652F656C6F7065735A
:1032B0002F50464531352F52494F5429290A00696C
:1032C000646C65006D61696E0000000000440040A0
:1032D000000002000300024002000240070700262F
:1032E0000048004000000400090C0240080C0240A5
:1032F0000707002700300140070002400600024097
:10330000050002400400024005000000001000001B
:1033100001000000003800400F0402400E0402408B
:103320000D0402400C0402400500000000400000B3
:103330000000000000000040FFFFFFFF0100000050
:10334000001C0000000C0040FFFFFFFF0800000011
:103350000032000002024750494F2043616C6C620A
:1033600061636B0A004F4E004F4646004750494F7D
:1033700020746F20554152542073616D706C65202C
:103380006170706C69636174696F6E0D0A004572DB
:10339000726F72207768696C6520696E6974696103
:1033A0006C697A696E67204C4544204750494F202C
:1033B0006173206F75747075740A004C4544204722
:1033C00050494F20696E697469616C697A6564203F
:1033D0007375636365737366756C6C7920617320B4
:1033E0006F75747075740A004572726F7220776819
:1033F000696C6520696E697469616C697A696E6768
:1034000020425554544F4E2055534552206173204D
:1034100065787465726E616C20696E746572727520
:1034200070740A00425554544F4E204750494F2063
:10343000696E697469616C697A6564207375636328
:1034400065737366756C790A004D657373616765A2
:103450002072656365697665642C204C454420695B
:10346000732025730A00000028020020430000009A
:10347000000000000000000000000000000000004C
:10348000000000000000000000000000000000003C
:10349000000000000000000000000000000000002C
:1034A000000000000000000000000000000000001C
:1034B000000000000000000000000000000000000C
:1034C00000000000000000000000000000000000FC
:1034D000232D302B20000000686C4C00656667458A
:1034E00046470000303132333435363738394142BF
:1034F000434445460000000030313233343536371E
:0C350000383961626364656600000000F9
:10350C00780B002000000000640300204000000045
:10351C000000000000000000BF320008C4320008A8
:10352C00010101012802002000000000B034000855
:10353C009034000870340008000000000000000007
:10354C0000000000000000006C34000800000000C7
:10355C00000000000000000000000000000000005F
:10356C00000000000000000000000000000000004F
:10357C00000000000000000000000000000000003F
:0C358C00000000000000000028210000EA
:04000005080004F1FA
:00000001FF
